:1000000012C0189518951895189518951895189563
:100010001895189518951895189518951895189578
:100020001895189518958FED8DBFC0ECE0EC4E2E0D
:10003000DD275D2EEEE7F0E0A0E6B0E0A89584B7FE
:10004000082E877F84BF88E1992781BD91BD8827CD
:100050008D933197E9F78FE289B980E082B988E121
:100060008AB966248FEF87BB18D1EEE1F7E012D290
:1000700017D216D2E1E0F0E0A0E698E330D3E2E355
:10008000F7E008D2A0E600D20BD20AD2E9E3F0E012
:10009000A8E991E024D3E4E4F7E0FCD1A8EAB0E0D9
:1000A000E8E9F0E06DD2EED1E4E5F7E0F3D1F8D184
:1000B000F7D1F6D1EAE5F7E0EDD1F2D1F1D1E0E602
:1000C000F7E0E8D1EDD1E2E7F7E0E4D1E9D1E2E809
:1000D000F7E0E0D1E5D1EAE8F7E0DCD1E1D1A6EA4A
:1000E00052D1A6EA0D911C91083E5DEF150709F06B
:1000F00006C0A5EA8C918F5F8C93A6EA0BD2009183
:10010000A5000C3009F001C01CC05F9BE8CF33E0B4
:100110009AD1A8EAB0E07ED2A9E90C93C1D10091AE
:100120009900013009F002C0D6D00BC0023009F0AE
:1001300002C0E3D006C0033009F002C002C001C013
:1001400099CFABD0E2E9F7E0A5D1AAD10CE310E05A
:10015000A8E94D9155272AD1AFE94D935C93AFE9BA
:100160000D911C9144E150E01CD1AFE90D931C931B
:10017000A0E6BCD2A3EA8C9381E08093A4004091D6
:10018000A3000091A400041710F009F071C0809141
:10019000A400E0E6F0E001E00A93AAE96DD2EAE902
:1001A000F0E0AAE9BFD1AAE98C91A1EA8C93AAE96F
:1001B000ECE9F7E0A1D209F002C062D053C000918F
:1001C000A1000F3381E008F480E08F930091A1003B
:1001D0000B3581E010F009F080E09F91892388239E
:1001E00009F402C060D014C00091A1000C3281E07B
:1001F00008F480E08F930091A1000A3381E010F0B1
:1002000009F080E09F918923882309F401C057D029
:1002100088E090E0ACE98D939C9391E0A2EA5FD1F5
:10022000ACE9B8D0A2EA0C9107FB0EF0F6CFACE92E
:10023000B1D091E0A2EA53D1C09AA2EA0C9107FB97
:100240000EF002C018D001C01BD0C09814D0ACE989
:10025000A1D0ACE90D911C91003050E0150709F0D8
:10026000E8CF0ED0A4EA8C918F5F8C9308F487CFEF
:1002700083CFF894FFCFAFE98D919C9121D1089560
:10028000AFE98D919C911CD1AFE98D919C9118D1D2
:10029000AFE98D919C9114D108958BE104D1EEE9E1
:1002A000F7E0F8D00895A1EA8C918F538C93ECE598
:1002B000F3E0A1EA8C919927A2EA29D10895A1EA55
:1002C0008C918C528C93E8E7F3E0A1EA8C9199270A
:1002D000A2EA1DD10895E2EAF7E0DCD0E1D0A0E681
:1002E00037E3B3D0DDD0A0E6CFD0DAD0E1E0F0E064
:1002F000A0E698E37BE7E5D10895E2ECF7E0CAD009
:1003000033E0A1D0A8EAB0E085D1A8E90C93009130
:100310009800053081E008F480E08F930091980008
:10032000043181E010F009F080E09F918923882357
:1003300009F407C0E9E3F0E0A8E991E07BE7B3D175
:1003400001C0DBCFADD0A8EAB0E0E8E9F0E018D119
:1003500099D0E4E5F7E09ED0A3D008957365061721
:10036000150B031D091F07180A1B04050819120D98
:100370000F020E1E0C1614134C736A2D2030383CDD
:100380003E3F2F272321ED91FC91EF5FFF4FFC9320
:10039000EE930895ED91FC91E150F040FC93EE93C3
:1003A000089508D03DD000FC10D0089503D01ED091
:1003B00001F8F9CF0024E89457FF02C009D06894EF
:1003C00000F80BD010F80124089502D009D0089548
:1003D000509540954F5F5F4F0895E89417FF08953B
:1003E000009510950F5F1F4F68940895352F242FA7
:1003F000E894452B11F468940895512F402F00275D
:10040000112780E1440F551F001F111F021B130B02
:10041000416018F4020F131F4E7F8A9599F70895D3
:10042000752F642F55274427FF93F1E1889405C069
:1004300010F4460F571F5695479517950795FA954F
:10044000B9F7FF910895A8EAB0E018D0883091F08C
:100450008D3039F03323C9F38D933A9563FE23D061
:10046000F4CF63FC04C08DE01ED08AE01CD0882746
:100470008C93089518D011973395E7CF5F9BFECFEB
:100480008CB10895A8EAB0E08D91882311F00BD0CB
:10049000FBCF08952CD0802D11F005D0FBCF08950F
:1004A0008DE001D08AE05D9BFECF8CB90895319735
:1004B000F1F70895689462F80895E89462F8089551
:1004C000EF93FF93EE27E82BE92B31F0E3E3F7E01E
:1004D0003197F1F70197D1F7FF91EF91089590309F
:1004E00029F08C91880F9A95E9F78C930895C89517
:1004F00031960020089591E005C092E003C094E099
:1005000001C098E0F4DF0D929A95E1F70895E80FA5
:10051000F91FF1CF82E001C084E099279D938A956D
:10052000E9F70895819104D08D938823D9F7089530
:10053000813618F08B3708F48F7D0895040F151F4E
:10054000261F371F0895000F111F221F331F089504
:1005500000951095209530950F5F1F4F2F4F3F4FFF
:100560000895019110810EC0019111912191308166
:100570000BC00191108117FF05C03FEF2FEF04C0A2
:10058000008111272227332737FF03C0E1DF8DE2E7
:100590008D93CF93DF93CF92DF92EF92AA24BB2467
:1005A000CC24DD24EE2440E2CAE0DD2755E093E3CD
:1005B0008881890F87FD9F7083FD907F891B8993B8
:1005C0005A95A9F7C0DFAA1CBB1CCC1CDD1CEE1C75
:1005D0004A9551F7E894EFE0FF2782910ED0EB3077
:1005E000E0F71EF068948A2D0CD088278D93EF9049
:1005F000DF90CF90DF91CF910895982F829501D011
:10060000892F8F70805D26F0803309F408956894F7
:100610008D93089500271127222733271DD08A3371
:1006200028F4803318F005D015D0F9CF0EF490CF10
:10063000089580538F93402F512F622F732F83DFA4
:1006400082DF7CDF80DF8F919927080F191F291F18
:10065000391F08958D910895E894FCDF8032E9F305
:100660008B32D9F38930C9F38D3211F46894F2CF0B
:10067000089588278D93089509919191992351F0B8
:100680008A95D9F7319781918D930A9519F088232E
:10069000D1F70895EECFE199FECFEEBB31960895E4
:1006A00091E001C092E07B3751F47FB7F894F3DF1B
:1006B0008D918DBBE29AE19A9A95C9F77FBF772712
:1006C0000895E9DF8D917B3729F48DBBE29AE19A99
:1006D0008823B9F77727089591E001C092E0DBDF26
:1006E000E09A8DB38D939A95D1F708958FEF839506
:1006F0009D919923E1F70895689401C0E894AF9320
:10070000BF938D9116F0919102C0F1DE902D891763
:1007100018F011F48823A9F7BF91AF9108955641BD
:1007200033544F20426561636F6E204B657965726B
:10073000000043757272656E74206D657373616736
:10074000653A200043757272656E7420537065655A
:10075000643A20002057504D00004D656E753A00F8
:10076000312E204368616E6765204D657373616744
:100770006500322E204368616E67652053706565A1
:100780006400332E20457869740028312D33293ACE
:10079000200052756E6E696E6720210020005B326A
:1007A0004A004E6577204D65737361676520283573
:1007B000352063686172732E206D61782E293A208E
:1007C00000004E6577205370656564202835202D24
:0C07D0002032302057504D293A20000004
:00000001FF
